:020000040800F2
:10000000501B0020CD000008F9300008F10F000857
:1000100000000000000000000000000000000000E0
:10002000000000000000000000000000C93D0008C2
:100030000000000000000000413300086143000898
:10004000DF00000800000000DF000008DF000008FB
:10005000DF000008DF000008DF000008DF00000804
:1000600000000000DF000008B9040008590500087E
:10007000DF000008DF000008DF00000800000000CB
:10008000DF0000086D44000800000000DF000008E9
:10009000DF000008DF000008DF000008DF000008C4
:1000A000DF000008CD3C0008DF00000885440008A0
:1000B0000D4500080348854600F0D6F80048004783
:1000C000494E0008501B00200844F0470448804770
:1000D00004480047FEE7FEE7FEE7FEE7FEE7FEE72F
:1000E00011440008B500000830B50B460146002059
:1000F0002022012409E00D46D5409D4205D31D462E
:100100009540491B2546954040191546521E002D25
:10011000F1DC30BD70B500242546002801DA012449
:100120004042002901DA01254942FFF7DDFFAC42D8
:1001300000D04042002C00D0494270BDF8B50024E8
:100140002546002904DA0E46012400214042B1412F
:10015000002B04DA1E46002352420125B34100F071
:1001600052F88C4617461E46AC4203D0002540424A
:100170008D41AC46002C02D0002657429E4161467C
:100180003A46334601B0F0BD10B5202A04DB0846DC
:10019000203AD040002110BD0B46D340D04020244F
:1001A000A21A91400843194610BD03460B439B0712
:1001B00003D009E008C9121F08C0042AFAD203E0DC
:1001C0000B780370401C491C521EF9D27047D2B202
:1001D00001E00270401C491EFBD270470022F6E786
:1001E00010B513460A4604461946FFF7F0FF2046AD
:1001F00010BD0321001D401E037812021A43491E40
:10020000F9D510467047F0B51FB40646002082B0FD
:1002100005464024019100901BE0019922460F46BB
:100220003046FFF7B1FF049A059B801A994110D31D
:1002300010461946224600F029F8361A8F410197D8
:10024000224601200021009F00F020F838184D417F
:1002500000902046641E0028DFDC019B00982946A0
:10026000324607B0F0BD0000064C0125064E05E001
:10027000E36807CC2B430C3C98471034B442F7D3C7
:10028000FFF71CFFD8580008F858000810B5202ABE
:1002900004DB0146203A9140002010BD914020230C
:1002A0009C1A0346E3401943904010BDF0B51C4C26
:1002B000A0684007C00F31D1206C1B4D82B2194895
:1002C0001A4903690120DE07002E0AD08A82184BE2
:1002D000184928469A4201D2012200E000220A6011
:1002E00012E09D4306D0144D9D4306D0134D9D430F
:1002F00006D009E00A83124806E00A84114803E0A8
:100300004A84114A528BCA834103490BA162A168F6
:100310000E4A1140091DA160024908610020F0BD8C
:10032000002401400000002000010020F412002001
:1003300098080000BC0000200000014000000244BA
:10034000000001C0000002C4A0F7FF1FE8FFFF7F0C
:10035000F0B51E4F85B03D691D4C6D1C3D61266892
:10036000A468029400966C466580019021816281A8
:100370000393386A01011748091800220B461046FA
:100380001C5CFF2C04D1401C1028F9D3002A17D084
:100390001022684600F012F9386AF861401C386291
:1003A0000001012109031030884201D90020386280
:1003B000F8680949401CF8604867002005B0F0BDA6
:1003C0001022684604F014FAE6E7000098000020C6
:1003D0008C58000800D0000874120020002911D0A9
:1003E0008268521882604368934200DCD21A00236C
:1003F0008361C368934201D1012343618260026932
:10040000521802610846704710B500231A4605E0ED
:10041000845C2407240FE318DBB2521C8A42F7DB0A
:100420001807000F10BD0000F0B50020174D012780
:10043000144B154C3F03E86017E0625A144EB24269
:1004400012D1EA680919521CEA604A882E69B24240
:1004500005D92A61E8614A686A61421C2A624988B2
:10046000994201D20B46A861401C0101B942E4D374
:10047000286A00011030B84201D900202862E868DB
:10048000F0BD0000FFC99A3B00D000089800002092
:10049000AA55000010B50421054800F0B0F8054841
:1004A00000218161C1610161C1600162084610BD26
:1004B00000D000089800002070B5234DE86A401C69
:1004C000E862224C20688006C00F11D02868296B92
:1004D00040182860296B28465830064600F058F826
:1004E00020206060B06900280AD00020286368726C
:1004F00020688005C00F02D001204002606070BDFE
:10050000304600F011FA12494A78A3585B085B00A4
:10051000A350F36832684E78D2180C4B0C33F2506B
:100520000A4B4A781B1DD658360C36040643D65063
:100530004978625801231A4362502863054881684C
:10054000802211438160D3E71402002000000240A2
:10055000A1580008003801400B49C86A401CC86215
:100560000A4802689204D20F05D001225203426069
:1005700000220A634A7201688903C90F02D001216F
:100580004904416070470000A802002000000240BA
:1005900010B5002910D0C26843685218934200DC9D
:1005A000D21A00234361C2608468944204D10122BC
:1005B00082618360C360C361084610BDF0B585B039
:1005C00016460D46074600F00FFB01200290002062
:1005D0000090019503A9684600F06EFA00247608A1
:1005E00007E060003A5A41190023012000F0BEFAEA
:1005F000641CA642F5D800F0AFFA05B0F0BD7FB597
:100600000D46044600F0F0FA00206A4631C203A904
:10061000684600F051FA00F09FFA04B070BD000087
:1006200006490020C861064801690422114301619E
:10063000016940221143016170470000301700201A
:1006400000200240064A0021D16106490A690223BE
:100650001A430A61486108694022104308617047E3
:10066000301700200020024010B5054B0022DA614F
:10067000044A1369012423431361018010BD000063
:10068000301700200020024010B50B4A0020D1682E
:10069000CB060A4904D5C86902231843C861102053
:1006A000D3685B0705D5CB6901242343CB610421C3
:1006B0000843D06010BD0000002002403017002029
:1006C00070B5044600F0A2FA0546104E0AE0601C20
:1006D00008D0002C04D000F099FA401BA04201D9A8
:1006E000032070BDF068C007F1D1F068800601D525
:1006F0002020F060F068C00602D4F068400703D5FF
:10070000FFF7C2FF012070BD002070BD0020024035
:1007100010B50E4C0020207220710D480078002882
:1007200000D10120A070E0700120C0020921C9069B
:10073000886288620749802088620A2000F0AEF94A
:1007400000F096F96061002010BD0000C800002094
:100750005700002000140048FEB5394D0121490220
:10076000284600F046FC00900120019040213548C9
:1007700000F03FFC044601210920C902C00600F038
:1007800038FC4021284600F034FC00262E4D00287D
:100790000BD0002013212D4A4901EF7803E01318F4
:1007A0005B181E75401CB842F9DB0098002802D186
:1007B00000F05EF9686128690127002814D10098CB
:1007C000002811D000F054F96969401A2049884284
:1007D0000ADBF9020922D20691617D21C9002F614D
:1007E000FFF798FC1B494884002C06D1E8680028D4
:1007F00003D01948018DC18406850198002817D0BF
:10080000002C17D0E86800280AD12F716E711348A8
:10081000026840218A4302606E7102680A430260E6
:10082000287A002808D12879002805D12F7102E004
:10083000002C01D12E716E71EC600020FEBD000015
:100840000004004800140048C8000020F40C0020F8
:1008500010270000340F00207414002000380040DE
:100860000A07120F01219140014201D00120704777
:10087000002070470A07120F01219140014201D068
:100880000120704700207047F8B50B051B0E254C62
:100890005B001C1909239B01E31800930523DB016E
:1008A000E618012307469B020A07E5180020120FED
:1008B0003B0003F0D7FF09060A0E12191D21282F4D
:1008C0002E00FF2928D800981BE0FF2924D8009883
:1008D00008E0FF2920D8B08A18E080291CD20F2018
:1008E00080012018808E11E0802915D2A88A0DE0A1
:1008F000402911D2B08E09E040290DD20B20800191
:100900000EE0808A02E0802906D2A88E1146FFF709
:10091000B1FFF8BD802901D30020F8BD0920C00136
:100920002018EEE7F40C0020C1688268914201DAD9
:10093000501A7047914202DC4269002A02D0406896
:10094000401A704780690028FBD000207047C268B9
:100950008168914201DA501A7047914202DC826943
:10096000002A02D04068401A704740690028FBD036
:100970000020704706490122896912030818010105
:10098000914201D3FF3801380249000140187047F5
:100990009800002000D00008F0B5334C4B001C1923
:1009A0000923DB01E5180B230246DB010020E318D5
:1009B000892A25D00EDC2C4F2C4B4E00F619F61848
:1009C000803A130003F04EFF091F1F152125292E21
:1009D000333A15008D2A3FD00CDC8A2A33D08B2A7B
:1009E00035D08C2A05D140293ADA0B208001201815
:1009F000808EF0BD992A03D0A12A01D0FE2AF8D119
:100A000080292DDA2EE00846F0BD102928DAB08AB8
:100A1000F0BD102924DAB08EF0BD102920DA0520AF
:100A2000C00108E008291BDA0F208001DFE7082950
:100A300016DA012080022018808AF0BD80290FDAA2
:100A40003420285EF0BD80290ADAA88AF0BD40294A
:100A500006DA0D208001CAE7402901DAA88EF0BD30
:100A60000020F0BD988EF0BDF40C00204002000084
:100A700010B5074A5068074B99695468A04201D0E5
:100A800050689969044A51430914401A10BD000086
:100A90001C00002000E000E05505000031B500F02A
:100AA000B5F8009C0546601C00D0641C00F0AEF850
:100AB000401BA042FAD338BDF8B5054623480F467F
:100AC000017E012601290BD0012101762868204CE6
:100AD000012807D02046FFF7F3FD002813D030E0AF
:100AE0000220F8BD2046FFF7EBFD002829D1FFF7D3
:100AF00097FD2046FFF7E4FD0646164801690422EB
:100B0000914301611DE00020C04338606C6812E031
:100B10002046FFF797FD0E48FFF7D2FD06460D4829
:100B20000169022291430161002E01D03C6008E07E
:100B3000012080022418A868696880024018A04239
:100B4000E6D80248002101763046F8BD3017002073
:100B500050C3000000200240034801698022114375
:100B6000016100207047000000200240F0B51FB472
:100B700005461A480024017E16461F46012907D063
:100B8000012101761648FFF79BFD002803D021E0E4
:100B9000022005B0F0BD012D1AD0022D18D0042579
:100BA00016E0220130463946FFF7EEFA81B201988D
:100BB00062001018FFF758FD0948FFF781FD094949
:100BC0000A69520852000A61002803D1641CE4B289
:100BD000AC42E6D3014900220A76DAE7301700205A
:100BE00050C300000020024005480169090605D5F0
:100BF000044941600449416000207047012070476A
:100C00000020024023016745AB89EFCD0148006811
:100C1000704700001001002002480168491C016073
:100C2000704700001001002010B50648016810222E
:100C300011430160002000F007F800F017F80020D1
:100C400010BD00000020024010B5044600F040F93D
:100C50007D21C900FFF748FA00F080FB0022214601
:100C6000501E00F025F8002010BD000008B50F4808
:100C70008169012211438161816911400091C2693A
:100C800001040A43C261C069002208400090114675
:100C9000501F00F00DF800221146901E00F008F8D9
:100CA00000221146501E00F003F808BD001002405B
:100CB00010B502F04FFA10BDF8B504460068364D85
:100CC000C00354D5E8690026C00007D4E8692904A8
:100CD0000843E861E8690840012600902F48016850
:100CE000C90511D4014608688A1510430860FFF74A
:100CF0008DFF074604E0FFF789FFC01B642823D857
:100D000026480068C005F6D5286A03210902084074
:100D10001FD062680A4082421BD0286A2A6A884330
:100D2000012109040A432A622A6A8A432A62286244
:100D3000C0070ED0FFF76AFF074607E0FFF766FF20
:100D4000C11B1748814201D90320F8BD286A8007DA
:100D5000F4D5286A032109028843616808432862A0
:100D6000002E04D0E869012109078843E861207852
:100D7000C00705D0286BA16880088000084328635D
:100D80002078800605D5286B10218843E168084348
:100D900028630020F8BD00000010024000700040F1
:100DA00088130000F8B5044644480E460068C007A2
:100DB000C00FB0420AD24148016849084900314396
:100DC00001600068C007C00FB0425CD120783C4F82
:100DD000800705D57868F0218843A16808437860CA
:100DE0002078C0073FD06068012813D039680228F6
:100DF00013D08907002946DA7968890889000143F8
:100E00007960FFF703FF0546606801280DD00228CE
:100E100017D024E039688903ECE78901EAE7FFF796
:100E2000F5FE411B2748814217D878680007800FDC
:100E30000128F4D117E0FFF7E9FE411B2148814268
:100E40000BD878680007800F0228F4D10BE0FFF779
:100E5000DDFE411B1B48814201D90320F8BD7868A3
:100E60000007800FF3D115480168C907C90FB142C7
:100E70000BD9016849084900314301600068C00787
:100E8000C00FB04201D00120F8BD2078400706D540
:100E90007868072109028843E1680843786000F018
:100EA0001DF87968084A0906090F515CC8400749CE
:100EB00008600020FFF7C8FE0020F8BD00200240B7
:100EC0000010024088130000C05800080C010020E8
:100ED00001480068704700000C01002010B513A005
:100EE0000FC888B06C460FC414A00FC80FC4174BAE
:100EF0005A680C20114601401548042902D00829DF
:100F000002D0144808B010BD9102090F6C46645C11
:100F1000D96A04AB0907090F595CD20303D5FFF75F
:100F2000E3F86043EEE70C486043EBE70203040597
:100F3000060708090A0B0C0D0E0F1010010203041E
:100F400005060708090A0B0C0D0E0F1000100240D1
:100F5000001BB70000127A0000093D00042204497A
:100F60000428086902D09043086170471043FBE7EA
:100F700000E000E015480168643101601448016830
:100F8000491C016013490868401C08601249134A53
:100F9000C868401CC860904216DB0020C86010483A
:100FA000816D491C8165016D491C0165416D491CBC
:100FB00041650C49088B002806D0401E80B208838A
:100FC000782801D97820088370470000200000208D
:100FD0001800002068000020E40000201027000016
:100FE00074120020A814002010B5FFF7C3FF10BD35
:100FF000FEE70069814301D000207047012070475F
:10100000332E303000000000FEB504460078D04D8D
:10101000C00746D068680007800F012807D06868BD
:101020000007800F022809D16868C00306D5286828
:10103000800336D5606800287ED032E001216068E8
:10104000090401280AD08A00002801D005280FD001
:101050002868884328602868904301E0286808438E
:1010600028606068002810D0FFF7D0FD064608E031
:10107000286810432860F1E7FFF7C8FD801B64284B
:101080006FD828688003F7D50BE0FFF7BFFD064651
:1010900004E0FFF7BBFD801B6428F1D828688003BB
:1010A000F7D420780126800700283BDA686800071B
:1010B000800F07D068680007800F022809D1686890
:1010C000C00306D42868800715D5E068012833D10D
:1010D00011E0E0680028286815D030432860FFF749
:1010E00095FD074604E0FFF791FDC01B0228C7D815
:1010F00028688007F7D52868F82188432169C90046
:10110000084328600EE0400840002860FFF77EFD9D
:10111000074604E0FFF77AFDC01B0228B0D8286814
:101120008007F7D42078000724D5E0690028686A92
:1011300010D03043686200E007E1FFF767FD074623
:1011400004E0FFF763FDC01B022899D8686A800796
:10115000F7D50FE0400840006862FFF757FD0746EB
:1011600005E09DE0FFF752FDC01B022888D8686AA1
:101170008007F7D4207804274007002860DA002091
:101180000190E869C00008D4E969B8060143E96143
:10119000E96901400120009101906E480168C9058C
:1011A00011D40168821511430160FFF72FFD0090F3
:1011B00005E0FFF72BFD0099401A642870D86548B8
:1011C0000068C005F5D5A06801280AD0002801D024
:1011D000052810D0286A400840002862286AB843D1
:1011E00001E0286A30432862A068002812D0FFF787
:1011F0000DFD00900AE0286A38432862F1E7FFF706
:1012000005FD0099411A5448814249D8286A80074F
:10121000F5D50DE0FFF7FAFC009006E0FFF7F6FCCD
:101220000099411A4C4881423AD8286A8007F5D47F
:101230000198002804D0E969012000078143E96191
:101240002078C00635D5606901280CD0401D686B38
:1012500023D038436863686B400840006863FFF739
:10126000D5FC064622E0686B38436863686B304300
:101270006863FFF7CBFC064604E0FFF7C7FC801B62
:1012800002285BD8686B8007F7D5686BF821884324
:10129000A169C900084368630BE0B8436863F4E7D9
:1012A0004CE0FFF7B3FC801B022847D8686B80072F
:1012B000F7D4206A002846D069680907890F0229F7
:1012C00043D001273F060228286805D0B84328608C
:1012D000FFF79CFC044633E0B8432860FFF796FC18
:1012E000064604E0FFF792FC801B022826D82868F7
:1012F0008001F7D4E86AE16A000900010843E86266
:10130000616AA06A084369683D2212049143084358
:101310006860286838432860FFF778FC044604E0DA
:10132000FFF774FC001B022808D828688001F7D555
:1013300009E0FFF76BFC001B022801D90320FEBD6A
:1013400028688001F5D40020FEBD0120FEBD00000C
:10135000001002400070004088130000094910B5D9
:10136000401E884201D9012010BD074C6061032155
:10137000081F01F0EFFE0020A0610720206100207F
:1013800010BD0000FFFFFF0000E000E010B50021ED
:101390000F4A0846516043009B18401C1981FF28E2
:1013A000F9DD002005230B4ADB014400A418E418F2
:1013B000401CA1821028F8DB00200923DB01440037
:1013C000A418E418401CA186FF28F8DD002010BDF9
:1013D0006C0A0020F40C002010B5402802DB00202D
:1013E000C04310BD10221143C200094B4000D21867
:1013F000C01858240D23A1529B010021C3189986BF
:10140000E300C0188186034800685065084610BD97
:10141000F40C00201001002070B504461E46383040
:10142000049D03F0F3FC20462A463146583003F071
:10143000EDFC002070BD000070B5104D0646014661
:101440002846FEF767FE0E4C2061FFF741FD294656
:10145000FEF74AFEA0600B48314600680546FEF7DD
:1014600043FEE0602A46002307480F21FEF766FE90
:101470002080206964306060002070BD40420F0011
:101480001C0000200C01002000004042034610B563
:101490000020024602E09C5C6040521C8A42FADB5B
:1014A00010BD0000F8B508460D460978552901D051
:1014B000252903D0012A01DD451C521E344F60242A
:1014C00079792B786143334C0919334C252B30D073
:1014D000A3685B1CA360CB695B1CCB61B978002956
:1014E0000FD0F97800290FD001292C4913D00723F8
:1014F0001B02C9180A7501462948FEF756FE00204E
:10150000F8700020C043F8BD2549264B55390A75AF
:101510000146224807E037235B01C9180A750146D6
:10152000204B1E482033C018FEF73FFEF878401CC1
:10153000E6E76E79802E06DDE068401CE060086A10
:10154000401C0862DDE7334608339A4208D2086A35
:10155000401C0862E068401CE0600220C043F8BD07
:10156000B11DFFF793FFA919897981420DD0206938
:10157000401C206179796020414306480818416A7F
:10158000491C41620320C043F8BD0020F8BD0000A3
:101590004C0000205C05002028030020F40C0020F3
:1015A00009140020D5060000F8B50E460446252093
:1015B000069F079D089920706270A670E3702771DE
:1015C0002F46002008376619372B1AD009DC1A4637
:1015D000303A130003F046F907261515262626177C
:1015E0002600612B0DD006DC382B0AD0412B08D009
:1015F000422B17D105E0622B03D0632B01D0642B63
:1016000010D1657102E06571002D03D02A46A01D3E
:10161000FEF7CBFDA91D2046FFF738FFB0710D2066
:10162000F0713846F8BD0000F1B584B0FFF7EEFA6E
:101630000446FFF71DFA524DE979002906D0297AB0
:10164000002903D0E968411A322905D8E9687D22CA
:10165000411AD200914263D9297A4A4A4A4E002956
:1016600061D06B79602701217B43F1506421516483
:101670006979491CC9B26971EA7A914208D9A96AA3
:10168000411AE962A862A979491CA971012169710D
:101690003E49098A3E4B6A793E499F5C0F709B1810
:1016A0005B784B706023384E5343F3588B700026A1
:1016B000CE700C71270A4F71270C8F71270ECF71D6
:1016C0006F46E8603878AF798008BF078000BF0FA9
:1016D00038436F463870002B4ED0EF2318403870D7
:1016E000009008232A4801930291412300211030E1
:1016F000FFF75AFF264902461031049802F0DCFB3E
:10170000687960214843204940184168491C41607C
:10171000C268E9688A1A4263C1606C63EE712E7216
:10172000002005B0F0BD696A491C69621A494B681E
:101730005B1C4B60697960238C4659438E4689193E
:101740000B695B1C0B614B695B1C4B61EF79002FD4
:1017500002D18F6A7F1C8F628F69BB4200D98B6177
:10176000032B85D900217346F150C8239364084B9D
:101770006246103B99547BE710231843AFE7000003
:101780004C000020741200205C050020A8140020EA
:101790004C0400205C08002028030020F7B50878DE
:1017A00086B00C46552801D0252802D0012A00DD3C
:1017B0004C1C424E62797079602104904843404944
:1017C0004518A868401CA860084680380390314638
:1017D0000B6BC968E778591A3346A0789B69303F8C
:1017E00000933B0003F03EF813420B17424242299C
:1017F000424242424242424242422C454200314928
:10180000A3790B542179A01D3223019200910290FB
:101810000021049A22E07161009A914200DDB161D9
:10182000284AA37913540020E9626861286B884232
:1018300000D229630120307218E00120F07115E018
:101840002048A179017010300078A0712179A01D85
:101850000192009102904223317900220398FFF710
:10186000A3FE02460399069802F026FB002009B069
:10187000F0BD7161009A914200DDB161114BA27916
:101880001A54114B181809239B01C018C2740F4831
:10189000008A0020E9626861286B884200D22963CF
:1018A0002046677A0A30FEF7A4FC617B0002000A3A
:1018B00009060843B90069188863BBE74C0000209B
:1018C0005C0500203C040020F40C0020A81400203B
:1018D000F7B515460C46FFF7CBF81A4E3063217862
:1018E0000020552903D1012D01DD641C6D1E3178C6
:1018F00000290FD00127F7712A4621460098FFF7EB
:10190000D1FD002805D137722A4621460098FFF7FD
:1019100045FFFEBD71780029FBD00B4E2A46B06B07
:101920002146401CB063009800F012F80028F0D166
:1019300006482A46406C30652146009800F080F841
:10194000FEBD00004C0000205C0500207412002049
:10195000F0B508460D460978552901D0252903D050
:10196000012A01DD451C521E297800231A4FDB4352
:101970001A4C252906D0A068401CA060386C401C79
:10198000386409E014496E79896C491C802E05DDA4
:10199000E068401CE060B9641846F0BD3346083387
:1019A0009A4206D2B964E068401CE0600220C0435D
:1019B000F0BDB11DFFF76AFDA9198979814208D0F0
:1019C0002069401C2061F86C401CF8640320C0436F
:1019D000F0BD0020F0BD00005C05002028030020C1
:1019E000F8B5FFF745F8134B1A69197900291FD08C
:1019F0005C7A1149002C05D07D20800148640020CC
:101A0000587215E00C4E0D4C851A8036A54204D94B
:101A10007D2292018A64012206E01219904207D9C0
:101A20007D2292018A6402228A67C8671869306041
:101A30000020F8BD4C00002074120020E02E0000B1
:101A4000F7B5087884B0552802D1012A00DD491C79
:101A50004A480268521C0260494B4A794878494E0C
:101A6000039335791C468034A84208D0FF2806D05D
:101A7000606C401C60640020C04307B0F0BDA84209
:101A800001D0FF2878D1306B009030610120707256
:101A90003B48CF7890380078372F6DD007DC303F47
:101AA0003B0002F0DFFE0669136969692169612F55
:101AB00062D004DC382F5FD0412F5DD11DE0622F52
:101AC0005AD0632F58D0642F56D14AE02C4B8F79CF
:101AD000A03B1F70887100983061881D09793223FE
:101AE0000192009102902EE00020097936230091A6
:101AF000019002460290012127E0214B8F79A03B03
:101B00001F70CF7A8B7A3F02DB19F361B37A887149
:101B100098004B720019078F8F72078F5B1C3F0A6A
:101B2000CF72876B3F0C0F73806B000E4873D8B277
:101B3000B0720A2801D30020B072881D09794223AF
:101B4000019200910290002229460398FFF72CFD94
:101B50000246E06B401CE0630399049802F0ACF984
:101B60000AE0CA798879120280180A7A497A12043E
:101B7000090651184018F06100207EE72803002074
:101B8000DC0400204C000020034610B50020024673
:101B900002E09C5C6040521C8A42FADB10BD30B50A
:101BA0000D46084609781446252901D0012030BD8C
:101BB000062C01D2032030BD611EFFF7E5FF291975
:101BC0002039C97F814201D0042030BD002030BDC2
:101BD000F8B51E460B465527069D079907704370BA
:101BE0008270C670044605712A46401DFEF7DDFA74
:101BF000691D2046FFF7C8FF014660194171A81D05
:101C0000052E02DA002E00D10020F8BDFEB51646E2
:101C10000F460546FFF7C3FF040014D06846047260
:101C20000420009002A90B4801910278401E01781F
:101C3000EE230948FFF7CCFF02460749284602F089
:101C40003BF92046FEBD32463946284600F006F8EC
:101C5000FEBD000085000020EC080020F7B5FA4822
:101C600086B04F7842688260421C15788E782D09C4
:101C700036072D01360F0B7935431570F34A029262
:101C800000780C460490874201D0FF2F77D121467F
:101C9000E6780931EE488C46332E72D028DCED49C7
:101CA000182E0A686CD012DC072E20D008DC002E1B
:101CB00065D0012E3ED0032E41D0052E7ED160E0AE
:101CC000112E7CD0162E7BD0172EF7D13FE2232E7B
:101CD000EED006DC192E74D0212E73D0222EEDD139
:101CE0008FE1242EE4D0312E4BD0322EE6D1BFE04E
:101CF000582E68D012DC542E66D008DC342E71D0F9
:101D00004F2E70D0502E6FD0532ED7D16EE2552E5D
:101D10006BD0562E6AD0572ED0D164E2304663384D
:101D20000421030002F09EFD09F0EFEE171D4A109A
:101D30004A154A00641D00930194012351E2C649EB
:101D4000182003E03946C7E2C4490C2001910090F5
:101D500005E0C348F6E1C24910395020F6E73346A2
:101D60003FE2E1790020B94A03E023185B7A13547B
:101D7000401C8842F9DBB54802F0D6FCA3E075E2CE
:101D8000EEE1A279617912028918E27989B2882B91
:101D90002DD0892B2FD08A2B31D0832B34D0842B7C
:101DA00037D0852B3AD0862B3DD0872B40D08B2B3C
:101DB00043D08C2B46D0FE2B1DD006E097E29FE14E
:101DC000AEE1EDE1C9E066E227E2A92B3FD0B32BFB
:101DD00041D0992B42D0A12B45D09C4810384018B7
:101DE00000925FE244E0F6E1F1E140E249E24900BD
:101DF00009189C483AE0490009189B4836E0490018
:101E000009189848203831E04900091895208000C9
:101E10002CE0490009189D20800027E0490009189E
:101E2000A520800022E049000918FD2080001DE067
:101E3000490009188B48A03818E049000918DD202E
:101E4000800013E049000918BD2080000EE0490021
:101E5000091886480AE04900854807E08548490096
:101E60000818001DBCE749000120C0060818B7E7A4
:101E7000A279617912028918E27989B2882B25D07A
:101E8000892B27D08A2B29D0832B2CD0842B2FD0A1
:101E9000852B32D0862B38D0872B3BD08B2B3ED056
:101EA0008C2B41D0FE2B45D0A92B47D0B32B49D04A
:101EB000992B4AD0A12B4BD06448103840180022EF
:101EC0006146FEF772F90020009024E149000918EC
:101ED000644840E04900091863483CE0490009189B
:101EE0006048203837E0490009189520800032E02A
:101EF000490009189D2080002DE049000918A520FF
:101F0000800028E0DFE1D2E1CEE149000918FD20A0
:101F1000800020E0490009185248A0381BE0490021
:101F20000918DD20800003E049000918BD20800069
:101F30000818C4E7490009184B48F9E7490009188F
:101F40004A48F5E749004A48F2E74900494802E0B3
:101F500049000120C0060818B2E7A279617912028F
:101F600089180922920189B2002B0FD0012B13D0BE
:101F7000022B1CD0032B20D0042B26D0052B2AD0DB
:101F8000062B28D0082B34D000202AE00B095B0058
:101F9000181833E0012024E00B095B00181811E049
:101FA0000A07120F012191400840F3D119E00A09F4
:101FB000520010180522D20120E00A095200101820
:101FC0000F2292018018808EEAE70A095200101849
:101FD0000122920212E0C90008184030007E40063B
:101FE000C00F69460873012003A9212301910090C5
:101FF000F7E00A09520010180922D2018018808ADD
:10200000CEE7A27961791202891889B2002B33D008
:10201000012B3AD0022B41D0032B48D0042B4FD0B8
:102020004022052B54D0062B52D0072B5BD000202A
:102030006946087300200090034803A9401C0191E1
:10204000027822237EE6000084000020EC080020B5
:10205000F40C00206C0A0020F2570008ACF7FF1FB8
:10206000107C0008B4040000B4050000B4060000B1
:102070005C050020740C00200B07090949000918B1
:102080001B0F9520E279800035E00B070909490014
:1020900009181B0F9D20E27980002CE00B0709092D
:1020A000490009181B0FA520E279800023E00B07E7
:1020B0000909490009181B0FFD20E27980001AE088
:1020C0000B0709091B0F49000918E2798D4812E036
:1020D000C90008184030018B9143E279D207520EB3
:1020E00011430183A6E70B07090949000918854830
:1020F000E2791B0F80300818194601F001FF99E7BB
:10210000002B05D0012B00D0DDE602F0AFF8DAE6B7
:1021100002F0E4F8D7E601907B48E378027811E614
:10212000A179607909024018E179784A80B2002BE0
:102130000AD0774C012B03D0764B9B8A002B03D01F
:10214000400000190091ADE040008018FAE7002A35
:1021500001D000200860002000901723019040E08B
:10216000002A01D000200860A17960790902401896
:1021700085B2E2790020684903E02618767A0E5489
:10218000401C9042F9DB6449284602F0DBFA00204B
:102190000934009001905C48039402781823D1E53B
:1021A000A1796079090241185A48C182818A0029BF
:1021B0000BD000218182574801F008FE00200090DA
:1021C0000190514819230278BCE50121F2E75148FA
:1021D0000383002002E04F49002008830090019013
:1021E000E3782A46AEE54B492020AFE5A179607936
:1021F00009024018494980B20A18E179121D78286D
:1022000001D3002105E00B18782B02D97821081A98
:1022100081B2C8B201920090A1E5A179607909026A
:1022200040183E4980B20B18E2791B1D782801D373
:10223000002205E01118782902D97821081A82B203
:1022400061461846FDF7B1FF0020009001902E482E
:10225000E378027839460298FFF7BAFC0246029901
:10226000069801F029FE2D4802F08CFA3CE02B483C
:1022700002F088FA0020009001902348552302784C
:1022800060E5244801F0A2FD0020009001901E4866
:102290005623027856E5032109022148FDF79EFFE7
:1022A0000020009001905AE51E481F4A4DE7A17991
:1022B000607909024018E17980B20D01FEF75AFBFE
:1022C000E9B2009127E7FEF7E5F8002000900190C1
:1022D0000D486523027835E50298FFF779FC024640
:1022E0000299069801F0E8FD002009B0F0BD022037
:1022F0006946087303A901200191EE232A46009044
:102300000499E9E71404000085000020008000081B
:1023100000A00008A8140020EC080020740C002085
:102320005C050020F40C0020F405000070B5FEF7F9
:102330007BF8164800F068FA154D164C6869A065E0
:102340001248816861658188491C81808088E064C9
:102350000E4801F03BFD2868206768686067A86840
:10236000A06701220C4B1146A06DFDF7F1FF20463E
:102370008030E9680160A9694160E9698160296983
:10238000C160296A0161002070BD0000A81400200E
:1023900098000020741200203930000008B504496C
:1023A0004A6902434A6149690140009108BD000041
:1023B0000010024008B50449CA690243CA61C969EC
:1023C0000140009108BD00000010024008B504491A
:1023D0008A6902438A6189690140009108BD000051
:1023E0000010024070B5094E04467618203E049D48
:1023F0000C34F17F0830102D03D00A50F07F0351C8
:1024000070BD0A51F17F0B5070BD0000CC53000825
:10241000044A51182039C97F42585208520042508C
:1024200070470000CC530008044A51182039C97F76
:10243000425801231A43425070470000CC53000811
:10244000044A51182039C97F425802231A43425086
:1024500070470000CC530008054B10B559182039BF
:10246000C97F435803242403A3431343435010BD9F
:102470009C580008054B59182039C97F001D0B587E
:102480001B0C1B0413430B5070470000CC53000877
:10249000054B10B559182039C97F4358034C2340C8
:1024A0001343435010BD00009C580008EFBFFFFFCE
:1024B000054B10B559182039C97F43588024A343D0
:1024C0001343435010BD00009C580008054B10B545
:1024D00059182039C97F43580324A402A343134346
:1024E000435010BD9C580008054B10B559182039B1
:1024F000C97F43582024A3431343435010BD000019
:102500009C580008054B10B559182039C97F43580D
:102510004024A3431343435010BD00009C580008BF
:10252000054B10B559182039C97F4358032424029C
:10253000A3431343435010BD9C580008F0B500233B
:102540003CE001249C40224037D04F680668144686
:10255000544365006519AE4367433E4306604E68C9
:10256000012E01D0022E05D18F6886686743AE43E5
:102570003E4386600F69C668AE4325467D432E43C1
:10258000C6604D68022D18D14D69FF2A09D8066A28
:10259000544354432201121B96436C432643066264
:1025A0000BE0140A22466243624362431401A61AF6
:1025B000446A6A43B443144344625B1C0A68144689
:1025C000DC40BED14A68012A01D0022A06D10A683D
:1025D000C968436893434A43134343600120F0BDF5
:1025E00010B5044601F0BCFA206001F09FFA60606B
:1025F00001F0AAFAA06010BD014610B50020002924
:102600000FD1104A116B8907890F01290AD00229BD
:1026100011D0032909D001F0A3FA01F087FA01F0E3
:1026200093FA10BD01F09CFA10BD11688907C90F1B
:10263000FAD0054810BD116A8907C90FFAD00120E8
:10264000C00310BD0010024000127A0010B50368EC
:1026500000225B06DB0F25D10CC98C681A434B683E
:1026600023431A43CB681A430B691A434B691A4335
:102670008B691A4303680C4C23401A43026042687A
:102680000A4B1A40CB681B0C1A430B681A43426072
:1026900001238A695B0308399A4202D1898C89B285
:1026A00001610122104610BD4000FFFFFBF0FFFF5B
:1026B000F0B50268194B1A4C984201D0A04203D1E0
:1026C0007025AA434D682A43164D174E174F98425E
:1026D0000AD0A04208D0164CA04205D0A84203D090
:1026E000B04201D0B84204D103242402A243CC68F2
:1026F000224302608A68C2620A888262984205D0D8
:10270000A84203D0B04201D0B84201D1097C016394
:1027100041690122114341611046F0BD002C014086
:1027200000040040004001400044014000480140D6
:102730000020004041680122D2029143416081683B
:102740000822914381607047FEB5044600680D463B
:102750000026C007C00F43D1E9686868AA6908432A
:1027600029691143084321681E4A1140084320602B
:10277000A86861680322120391430143616068699C
:10278000A168121191430143A1601748844203D10B
:102790000020FFF731FF06E01448844220D168464C
:1027A000FFF71EFF029800281AD02968002917D0C9
:1027B0000126AA69F3039A420CD140004A08801806
:1027C000FDF792FC0A4980B201400007420F0A431C
:1027D000E26005E04A081018FDF786FC80B2E06070
:1027E0003046FEBDF369FFFF003801400044004061
:1027F000F0FF000010B580220249FDF7D6FC002052
:1028000010BD00000C580008F0B5154A0021551401
:10281000144C154F0CE0D65ABE4208D19B185B8869
:102820006668B34203D90AC44B1C2360083C491CA8
:102830004B01AB42EFD321680123002905DB49019D
:102840008918202201F0C2F900E08380A0684001CD
:102850002030A84201D90020A0600020F0BD000077
:1028600000C8000898000020AA5500001FB50B46BC
:10287000024604A1684601F0E1FF0146684601F006
:1028800033F91FBD201B5B25643B25644800000015
:1028900010B50120FFF782FD00210A2000F038FC6E
:1028A0000A2000F02BFC00210B2000F031FC0B2053
:1028B00000F024FC10BD0000F0B5012087B04004FA
:1028C000FFF76CFD01208004FFF768FD0120C004C4
:1028D000FFF764FD01208005FFF760FD0126C020A1
:1028E000002403256A46049631C20927FF0669467B
:1028F0003846FFF723FE8020694631C169463846D5
:102900000494FFF71BFE9320000100900394694696
:102910000196029504943846FFF710FE3002B86124
:1029200068026A46049631C269463846FFF706FED9
:1029300029486A46049631C269462848FFF7FEFDD9
:102940002748009003946946019602950494234811
:10295000FFF7F4FD072040030090029403946946BA
:10296000019604941F48FFF7E9FDF0206A4604969B
:1029700031C269463846FFF7E1FD3002B8614000D8
:102980006A46049631C269461448FFF7D7FD4020D5
:102990006A46049631C269461348FFF7CFFDF0023C
:1029A000009069460196029504943846FFF7C6FDEB
:1029B0008020009069460196029504940A48FFF72A
:1029C000BDFD40206A46049631C269460348FFF7C0
:1029D000B5FD07B0F0BD000007040000000400488A
:1029E000C0FC0000000800480014004808480749DF
:1029F00001600849016004214160074A8260C168A2
:102A00004907FCD10261054901607047CCCC000048
:102A10000030004055550000FF0F0000AAAA00003A
:102A2000F0B591B0282106A8FDF7D8FB182168461B
:102A3000FDF7D4FB01200003FFF7C8FC0120800450
:102A4000FFF7ACFC00240825022603270394049416
:102A50006A460594E0C269462248FFF76FFD1020E0
:102A600069460394C1C101200490694605941D483C
:102A7000FFF764FD2020039404946A460594C1C2C4
:102A800069461848FFF75AFD0021192000F040FB65
:102A9000192000F033FB0720000208900120069463
:102AA0000A9040020B900994802007940E940D9098
:102AB00007200D4C0F900C9506A92046FFF7C6FD88
:102AC00060681021884360606068A8436060606847
:102AD0000902884308436060206840210843206061
:102AE00011B0F0BD000400480030014010B586B0C0
:102AF00014216846FDF772FB1020FFF75BFC0021F4
:102B0000112000F005FB112000F0F8FA2F20694693
:102B10000880002001900848084C02902046FFF7EA
:102B2000C7FD2068802188432060E06801210843B8
:102B3000E06006B010BD0000E70300000010004098
:102B400070B501208EB08003FFF740FC03204002E7
:102B500007900220089003200024099001250920F5
:102B60000A9407A90C950B94C006FFF7E7FC3A4EB0
:102B7000102202213046FFF78BFC00220221304652
:102B8000FFF76AFC002202213046FFF7ADFC00226D
:102B900002213046FFF7B6FC802202213046FFF7C3
:102BA00087FC002202213046FFF7BAFC00220221F6
:102BB0003046FFF78BFC002203213046FFF768FC0C
:102BC000002203213046FFF747FC00220321304654
:102BD000FFF78AFC002203213046FFF793FC802296
:102BE00003213046FFF764FC002203213046FFF743
:102BF00097FC002203213046FFF768FC00211B20D0
:102C000000F086FA1B2000F079FA14486946006843
:102C10000090019402940394059406940C20104CA7
:102C200004902046FFF790FD606829050843606026
:102C30006068490003225205904308436060A06821
:102C400049120843A0602046FFF774FD206828431E
:102C500020600EB070BD0000000002403400002073
:102C60000038014070B58EB01C216846FDF7B6FAF9
:102C7000182107A8FDF7B2FA012464042046FFF7E3
:102C800099FB2046FFF78AFB0E2007900220089050
:102C9000032001250990002409200A9507A90C9515
:102CA0000B94C006FFF74AFC414E10220421304627
:102CB000FFF7EEFB002204213046FFF7CDFB002298
:102CC00004213046FFF710FC002204213046FFF7B4
:102CD00019FC802204213046FFF7EAFB0022042180
:102CE0003046FFF71DFC002204213046FFF7EEFBC3
:102CF000002205213046FFF7CBFB0022052130469C
:102D0000FFF7AAFB002205213046FFF7EDFB00226A
:102D100005213046FFF7F6FB802205213046FFF7FC
:102D2000C7FB002205213046FFF7FAFB00220521F0
:102D30003046FFF7CBFB00211C2000F0E9F91C20F6
:102D400000F0DCF9A61EFF21304600F0E1F9304624
:102D500000F0D4F91748EE03006800900194029443
:102D600003940C2004AA51C2134C69462046FFF775
:102D7000EBFCA06821140843A060A068B043304376
:102D8000A06020681F21490588430843206020680F
:102D90004911884308432060A068A1140843A0603B
:102DA0002046FFF7C7FC2068284320600EB070BDA6
:102DB00000000240380000200044004000B50846F2
:102DC000042A02D80020C04300BD01787F2902D91F
:102DD0000120C04300BD41784906490E1F2902D990
:102DE0000220C04300BD114601F0DAFF0028F9D0EF
:102DF000042000BDF7B588B00F460A9A0898FFF77F
:102E0000DDFF0690002803D00020C0430BB0F0BDCA
:102E1000B6483A780078394682427DD18C784A7833
:102E2000CB78B98824024DBAB1491C4308704A7066
:102E300001200790200521070226000E090F13002C
:102E400001F010FD119E0A47859FB7D59E9E9E9E5C
:102E50009E9E9E9EE1F39E00E81DC008A44903903B
:102E6000887000202FE0002000900120019002983F
:102E70000027C00004901CE02005000E42009D4881
:102E800021071218092080011018090F808EFDF704
:102E9000E7FC002803D001990098084300900198AE
:102EA000641C4006000E7F1CA4B20190082F03DAB8
:102EB0000498C019A842DFDB8D49029A009889184E
:102EC000C8700298401C039902908842CBDB7618A8
:102ED00055E0E81DC008864903908870002031E065
:102EE000002000900120019002980027C00004906B
:102EF0001EE02005000E42007E482107121809201E
:102F000080011018090F808AFDF7AAFC002805D05F
:102F100001990098084300E0E5E000900198641CE6
:102F20004006000E7F1CA4B20190082F03DA04981B
:102F3000C019A842DDDB6E49029A00988918C87052
:102F40000298401C039902908842C9DBBFE76800E1
:102F500067498446887000200EE021184A006549C0
:102F6000470052180921C9015118898E604A0B0A7D
:102F7000BA18D3701171401CA842EEDB17E0761C22
:102F800087E068005A4A8446907000200DE02118BE
:102F90004B00584947005B18092189015918898A53
:102FA000BF180B0AFB703971401CA842EFDB664466
:102FB000E5E7002D12D0FF221202954207D1420010
:102FC0004C4812189D208000101800F091FF3946DF
:102FD00047480A9AFDF7E9F80A9E7FE04200454813
:102FE00012189D208000101800F042FEEFE738799B
:102FF0007979000208433F49620052180921C9014A
:1030000051188886E3E7E81DC008394903908870A5
:10301000002030E03818C079009001200190002095
:1030200005900298C00004901FE036E02005000ED5
:1030300042003048210712189D20090F8000101807
:10304000009B019A1A4202D000F052FF01E000F00A
:103050000FFE0198641C4006000E01900598A4B272
:10306000401C0590082804DA049805994018A842E5
:10307000DCDB0298401C039902908842CADB1C48A2
:10308000B9788170F978C1703979017179794171B4
:10309000361D0698002814D025E000200EE04100DF
:1030A000C919CA79097A12020A4321184B00114939
:1030B0005B180921C90159188A86401CA842EEDB19
:1030C000DDE70798002809D0B1B2094801F068FE91
:1030D00007498855000A89194870B61C32460449C8
:1030E000089800F0E9FE002090E600009000002023
:1030F000EC090020F40C002070470000C106C90E46
:1031000001208840014908607047000000E100E0AC
:103110008307FF22DB0E9A408907090E9940002899
:103120000BDA0007000F0838830808489B001818BE
:10313000C36993430B43C3617047830804489B00F2
:103140001818036893430B430360704700ED00E0D9
:1031500000E400E08307FF22DB0E9A408907090E96
:10316000994000280BDA0007000F08388308084848
:103170009B001818C36993430B43C36170478308CE
:1031800004489B001818036893430B43036070477F
:1031900000ED00E000E400E0F3B5074681B0002058
:1031A00000903D78FF206E07EC08760FE40001F0F8
:1031B00039FE802C01D20020FEBD324601265C493A
:1031C0005C48130001F04EFB0805313539898D91BB
:1031D000A1B057490978002903D0554949788C4254
:1031E00020D18188544F491C81803D70504D302141
:1031F000A87808437870E8780843B8703520F870EC
:1032000004213846FDF700F93021084338710D20BC
:103210007871112001F006FE0621384600F016FEF6
:103220006C702E704248067162E0C188491CC180F2
:103230005EE00189491C01815AE00A78002A02D027
:103240004A78A24201D00E7152E042893849521C9C
:1032500042810020CA780EE04100C9194B78897874
:103260001B010907090F5B1834490C181321490188
:1032700061180B75401C2E4C9042EDDB2E4A00204D
:1032800015702E4F0FE009213B1889015B18197D3D
:103290000D094100891830354D701B7D1B071B0F30
:1032A00030338B70401CA1788842ECDB0806C00DDF
:1032B000401CC1B22048FDF7A7F830210843A1788F
:1032C0001D4A49008A1850700D209070C91CC9B25F
:1032D000194800F0BBFD26710AE08189491C8181F3
:1032E00006E0C189491CC18102E0018A491C0182B2
:1032F00002980007C10E1148091813208001081810
:10330000818C491C81840098FEBD428A521C4282F5
:103310000878002897D04878A04294D10120C002B4
:103320000922D20690618EE7028B521C02838AE743
:10333000C8000020B4110020C8140020F40C0020A4
:1033400010B501200449C006486004480168491CC2
:10335000016000F005F810BD00ED00E03000002035
:1033600070B50E4801780024002905D004700C487F
:1033700001780C48FFF710FF0B4DE86F00280BD0C9
:103380000A4E0B4902203268FEF7A2FA3460EC675D
:103390008021074801F040F970BD0000E0000020E6
:1033A000E100002008150020A802002040000020B5
:1033B000BC03002010B50648054B00780021403BB7
:1033C0005A1840325478491C14700F29F8DB10BD8C
:1033D000340D002010B5084C084B01220221A06DCD
:1033E000FCF7B6FF064800F0F1FCE06D401CE0651C
:1033F000A06D2066002010BD74120020393000003E
:10340000A81400200248C16D491CC1650020704706
:1034100074120020F3B5FA4D85B0286800286FD0EB
:10342000686800281CD000220D21082000F080FDD3
:1034300000221146082000F07BFD012211460820E1
:1034400000F076FD00200146EE4A13184033401C80
:1034500019701028F8DB00260121144640347BE265
:103460000122E1E7B2000598059B805CD7187A78C5
:10347000019201257B8800931B2873D012DC024641
:10348000030001F0EFF91B5C7272727272723E3EC1
:103490003E3E3E3E5C5C5CA7A7A73E3EBEBEBEBEB7
:1034A000BEBE5C00342870D011DC01461C390B0014
:1034B00001F0D8F918A7A7A7A7A7A7A7A7A7A7A705
:1034C000454545454545454545454545F7453A2822
:1034D00073D008DC014635390B0001F0C3F905E271
:1034E0006E56E26E3000DC2804D004DC3B28EFD0BE
:1034F000C82824D120E1DD28FCD0FA28F9D11BE12D
:1035000033E2D01F030001F0ADF90E080A10181BBA
:103510001D1A1A1A1A1A1A20261A207C4AE0FFF7D6
:1035200049FF00281FD0207C3AE0FFF743FF002826
:1035300016D1207C002813D125E000F0C3FAF5E174
:103540002078F7E7FFF736FF1DE0207C00280AD03F
:10355000002905D007E0207C002804D1002902D0F2
:10356000012010E04DE000200DE0130001F07AF999
:10357000070C050E111B262E0C0000F0A3FA009973
:103580000198FDF781F92074D0E11AE100F09AFA70
:103590000CE0207C0028E6D000990198FDF774F932
:1035A0000028E0D0DCE7207C0028DCD000990198DE
:1035B000FDF76AF90028D6D1D2E758E1207C00282F
:1035C000CED100990198FDF75FF9B3E7207C002880
:1035D000ECD0C5E7102804D0112804D0122AAED1AF
:1035E0000AE0227C03E0207C0028A8D00122009978
:1035F000019800F09DFC99E1207C00289FD00022DA
:10360000F5E715383D79030001F02CF9120A12157F
:10361000181B0F1E3C4C5B6A2D798185898D7D942A
:1036200000F050FA13E0207484E000F04BFA1DE043
:1036300000F048FA29E000F045FA36E000F042FADE
:1036400042E000F03FFA4EE0207C002870D028468F
:103650000099FDF7A1F90546F9887879FDF79CF9FD
:10366000854263D064E0207C002861D02846009920
:10367000FDF792F90546F9887879FDF78DF98542CD
:1036800054D155E0207C002852D028460099FDF7FF
:1036900083F90546F9887879FDF77EF9854245DB9F
:1036A00046E0B1E0207C002842D028460099FDF792
:1036B00073F90546F9887879FDF76EF9854235DCAE
:1036C00036E0207C002833D028460099FDF764F9C5
:1036D0000546F9887879FDF75FF9854226DD27E010
:1036E000207C002824D028460099FDF755F905468E
:1036F000F9887879FDF750F9854217DA18E0207CCF
:10370000002813D1A3E7207C00280FD1AEE7207C4E
:1037100000280BD1B9E7207C002807D1C5E7207C21
:10372000002803D1D0E7207C0028DCD001207AE7F4
:10373000002078E70225F9E03F791546C8280DD02A
:10374000DC2823D0DD282AD0FA28F3D12D48E9003F
:1037500008184030007EC0062AD508E02948E90054
:1037600008184030007EC00601D4002121E0207CF2
:10377000002822D038460099FDF70EF90146284668
:1037800000F07EFA284600F0F5F84CE71D48E90005
:1037900008184030007EC006E9D4012109E019482C
:1037A000E90008184030007EC006E0D4022100E0A5
:1037B00003212846FDF710FED9E7284600F0AEFDAC
:1037C000E0E73F790225342802D0372816D108E0F7
:1037D000207C002812D038460099FDF7DDF8401C07
:1037E00007E0207C002809D038460099FDF7D4F87E
:1037F000401E02463846009900F012FC96E0000098
:103800006C0A0020F40C00203D7979790291F98846
:103810000191332814D035281BD038288AD1207C38
:10382000002887D00298FDF7B7F807462846009988
:10383000FDF7B2F83A1A0199029800F0F1FB79E726
:10384000207C0028FBD028460099FDF7A5F8024609
:10385000F1E7207C0028F2D028460099FDF79CF87B
:10386000054601990298FDF797F82A18E3E73A7997
:1038700079790291F9880191797A03917D893628C5
:1038800006D0392812D03A281FD03B284DD131E03C
:10389000207C002849D010460099FDF77DF80746A6
:1038A00001990298FDF778F83A180CE0207C00287E
:1038B0003BD010460099FDF76FF807460199029832
:1038C000FDF76AF83A1A29462CE0207C00282CD013
:1038D00010460099FDF760F807B201990298FDF7CC
:1038E0005BF800B247433A462946039800F098FB3C
:1038F0003A1416E0207C002817D010460099FDF7F6
:103900004BF807B201990298FDF746F801B2384624
:10391000FCF700FC02B20F462946039800F080FB3A
:103920003A46691C039800F07BFB032530114100E7
:103930000F48012308183107090F02898B401946E7
:10394000114000D00121277C0830002F01D01A43FC
:1039500000E09A43028076190698864200DA81E5F3
:1039600003494868401C4860002007B0F0BD0000D3
:103970006C0A0020FEB50746402802DB0020C04349
:10398000FEBD2C48F9000E1800964036348BE10637
:1039900001D40020FEBDA1063CD561063FD42649D6
:1039A000096800980A25406D0190081AA1070FD0F8
:1039B000A107890F012905D0022905D0E143890714
:1039C00005D005E0642503E07D25ED0000E01B4DFA
:1039D000A84224DB2946FCF79DFB014615487A00E6
:1039E00012180B20800110188446808E019B40180D
:1039F00069435B18009980B24B650D21890151180C
:103A0000898E814203D8084640210C4334836146A5
:103A1000888604E0600602D5402084433483307EEB
:103A2000B9B24006C20F052000F082FA307E40068F
:103A3000C00FFEBDF40C0020100100201027000074
:103A4000F7B50446FCF783FF054602992068A942B2
:103A5000A16806DC4018029A0199FCF7A6FB0299BE
:103A600019E040182A460199FCF79FFB2946204699
:103A7000FCF7B4FC2046FCF76AFF06460298471B99
:103A8000B7420DDCA16820683A46401801994919EF
:103A9000FCF78BFB39462046FCF7A0FC0298FEBDE4
:103AA000002E0CDDA16820683246401801994919A2
:103AB000FCF77BFB31462046FCF790FCAD1928460D
:103AC000FEBD0000074A0F2011183F235B5C403108
:103AD000401E0B700028F7DC02494031087C08705A
:103AE00070470000F40C002010B50C460A46014651
:103AF0000348FFF7A5FF00F077FD204610BD00004A
:103B00006C02002010B50C460A4601460348FFF738
:103B100097FF00F069FD204610BD00006C020020F8
:103B200010B50C4600F0C8FD204610BD0449496898
:103B3000F0221140034A0909515CC8407047000057
:103B400000100240C058000803494968034A49056B
:103B5000490F515CC840704700100240D05800081F
:103B600010B5074841680C200140064805D00429DB
:103B700004D0082901D100F009F810BD024810BD99
:103B80000010024000127A00001BB70010B50C4C68
:103B90006168012212040B48114002D0914200D109
:103BA0000948E16A0907090F491CFCF79DFA616899
:103BB0000F2292041140890C891C484310BD00005B
:103BC0000010024000093D00001BB70070B5D4177B
:103BD000A40F0023A418A51003E09C000E59065161
:103BE0005B1C9D42F9DCD40F6B00A418651003E048
:103BF0005C000E5B06535B1C9D42F9DC104670BDF9
:103C00000920C006006901090F20884370470000A1
:103C1000F8B5002384468025DB4312480024214662
:103C20002A464A43121817880F4EB74209D17E26FA
:103C3000B75A0E4EB74204D15288A24201DD0B465C
:103C40001446491C0829EBDB082B06D26B431918D4
:103C500080226046FFF7BAFF02E06046FEF7CAFD29
:103C60000020F8BD00C00008AA550000A55A0000B9
:103C70000B0702881B0F012199408A43028070477D
:103C800030B5402802DB0020C04330BD0D4CC200DF
:103C900013191A464032157EAD0611D440000019A2
:103CA0000D24A4010419A1860B240021A4010019EC
:103CB0008186054800685865108B202108431083D1
:103CC000002030BDF40C00201001002010B500F0E1
:103CD00001F810BDF0B52D4FB868C007C00F4DD02A
:103CE000F8682C4DC4B22A48C16A491CC162018DD2
:103CF000491C01852878002802D1204601F092F85D
:103D000028780026002819D12448234902788C54A9
:103D10000178491C01700D2C10D10446007801F087
:103D200081F820781E4908701E490120087026700D
:103D30001D48067001201D490007486028780028AA
:103D40001CD01B490878401C08701A48026B521C92
:103D500002630878184A1278904210D30120C002FA
:103D60000921C90688612E701449012008700E4986
:103D700008700A480670124980208862F0BD114818
:103D80000978405C387301F04DF8F0BD0030014017
:103D900074140020D000002008150020CD00002061
:103DA000E1000020E0000020CC00002000ED00E059
:103DB000CF00002074130020CE000020E20000207D
:103DC00000140048E81400207047000070B51A4C39
:103DD0006168491C616019490180A18841801849C6
:103DE000CA6C8280496D8160112181831549C1832C
:103DF000A1684A011449511800250B462A469E5CC9
:103E0000FF2E04D1521C202AF9D3002D10D02022DD
:103E1000FCF7D4FBA0682060401CA0604001012199
:103E200089022030884201D90020A060002070BDA6
:103E3000202200F0DDFCEDE798000020AA550000EC
:103E400074120020A55A000000C8000870B503468F
:103E50000E460807C10E1348002509180520C001A9
:103E60000818818A104C491C8182207A002817D1B9
:103E7000324619460D48FCF798F9A6710020E0710A
:103E80000A48E179405C0A4908730121217200F077
:103E9000C9FF08498020886100010921C90688629C
:103EA000284670BDF40C0020C8000020E814002053
:103EB000003001400014004810B514460A4601289D
:103EC00002D0022806D00DE021461046FFF71AFE68
:103ED000054804E021461046FFF722FE0348816FA3
:103EE000491C8167204610BD14020020A802002052
:103EF0000B0702881B0F012199400A43028070477B
:103F00000907090F01238B400188002A01D01943BA
:103F100000E09943018070470907090F01238B4096
:103F20000188002A01D0194300E0994301807047BD
:103F300070B50B051B0E204C5B000D071C192D0FD7
:103F4000030000F08FFC09060B14191E22272C31E8
:103F50003600FF292DD89520800003E0FF2928D8BE
:103F60009D20800020182946FFF7D6FF21E0FF2979
:103F70001FD8A5208000F5E780291AD2FD208000F7
:103F8000F0E7802915D20D48ECE7402911D2AD2089
:103F90008000E7E740290CD2B5208000E2E78029C5
:103FA00007D206482030DDE7802902D2034880305E
:103FB000D8E7002070BD0000F40C002014040000BD
:103FC0000121C903034A002801D091627047916121
:103FD000704700000008004801218903034A0028B7
:103FE00001D091627047916170470000000800485D
:103FF0000121C903034A002801D0916170479162F1
:10400000704700000008004801214903034A0028C6
:1040100001D091627047916170470000000800482C
:10402000F0B5304C4B001C190923DB01E6180B23BB
:10403000DB01E51892B28A283DD00EDC294F4B00F7
:10404000DF1909239B01FF188338030000F00AFCE5
:104050000714181C21262D46480099283ED006DC5E
:104060008B282CD08C2831D08D2839D133E0A12851
:1040700034D0FE2834D131E0102931DABA822FE071
:1040800010292DDABA862BE0102929DA0520C00183
:1040900008E0082924DA0F20800114E008291FDA3B
:1040A00001208002201882821AE0802918DAB28664
:1040B00016E0AA8614E0802912DAB28210E04029C4
:1040C0000EDA0D2080012018828609E0402907DAE7
:1040D0000B208001F7E7402902DAE8E78029E8DBD6
:1040E0000020F0BDF40C0020F0B58DB0002500F0EC
:1040F00015FEFCF7BDFC059010213A4800F070FE5B
:104100000790FCF7B5FC04901021364800F012FE31
:104110000690FCF7ADFC03901021324800F028FE19
:104120000190FCF7A5FC064610212E4800F038FE51
:104130000090FCF79DFC2C4A04469068012108433E
:104140009060881E106129481061264B0021585C40
:104150001070491C1029FADB1768FCF789FC0B90DA
:104160000199009802970190214F0091781921A19F
:10417000069B079A00F062FB45190B98A11B001BD8
:1041800001910290039A04990398B21A431A00927B
:1041900008460599421A781920A100F04FFB4419EE
:1041A00008A8FEF71DFA26484268012000040240D4
:1041B0003819134623A100F041FB0419381926A130
:1041C000089A00F03BFB01193846FFF78DFC0121EE
:1041D0000D20FEF74BFB24490320886000200DB022
:1041E000F0BD0000BC5300080030024001A00000F8
:1041F000140100200D0A435243202025303458205A
:1042000020253034582020253034582020253034C3
:10421000582020253034580D0A00000074696D655F
:10422000202530346420202530346420202530348B
:10423000642020253034642020253034640D0A00A9
:10424000001002404D61696E536F757263652025E1
:1042500078202564200D0A00737973636C6B202528
:1042600064200D0A000000000000002030B500218D
:10427000174D0846696042005219401C1181FF2801
:10428000F9DD00200522134CD20143001B199B18B5
:10429000401C99821028F8DB00200922D20143003B
:1042A0001B199B18401C9986FF28F8DD002010225E
:1042B000C100091940310B8B401C93430B834028EC
:1042C000F6DB0120044928604882002030BD000050
:1042D0006C0A0020F40C0020A814002010B5002166
:1042E0000C48092201600C4B084692014400E41876
:1042F000A418401CA1861028F8DB0020012292029D
:104300004400E418A418401CA1820828F8DB00200F
:1043100010BD00006C0A0020F40C002010B54028ED
:1043200002DB0020C04310BD0B4BC100CA18114670
:1043300040310C7EA4060DD54000C0180B2300248C
:104340009B01C0188486054800685065088B2022B0
:1043500090430883002010BDF40C002010010020C1
:1043600010B5FCF759FCFCF73FFE10BD70B594B0DA
:1043700030216846FBF732FF0024022501260E9407
:10438000E8030990009605200F94C0040D9401964F
:104390000A900C9408950B956846FCF735FE0028AA
:1043A00003D0862115A000F047FA07200C900E9448
:1043B00001210D950F940CA8FCF7F4FC002803D004
:1043C00092210EA000F038FA109610A81296FCF771
:1043D00073FC002803D0A12108A000F02DFA4B2087
:1043E0008001FCF7BBFF0420FCF7B8FD002211465A
:1043F000501EFCF75DFC14B070BD00002E2E5C4317
:104400006F6D4C69625C5372635C4253502E630063
:10441000134801680122114301604168114A1140AB
:1044200041600168104A1140016001680122920454
:104430009143016041683F22120491434160C16A87
:1044400009090901C162016BFF2214329143016322
:10445000416B4908490041630021816070470000B9
:10446000001002400CB8FF08FFFFF6FE0448016987
:10447000C907C90F02D00121C9430161704700007B
:104480000010004070B51B4CE0691B498006C00F4E
:1044900011D01A4A01201060194A10600869401CA6
:1044A0000861A28C4868401C4860174B154D18687D
:1044B0002A54401C1860E0690007C00F04D008208F
:1044C0002062C869401CC8612068C006C00F07D0C0
:1044D000E069C006C00F03D01020206200F03CF855
:1044E000E0694006C00F03D04020206200F074F85D
:1044F00070BD00000038014014020020440000207C
:10450000480000203C0300203C00002010B5104C67
:10451000E069E0690007C00F05D0082020620D485F
:10452000C169491CC1612068C006C00F07D0E0699D
:10453000C006C00F03D01020206200F09DF8E06993
:104540004006C00F03D04020206200F0E5F810BD07
:1045500000440040A80200200548416A491C41620D
:1045600004490968002901DD0121C1677047000085
:10457000140200203C000020F8B5144D0C460646FD
:1045800002212846FDF744FF10200090104B3246D0
:1045900002212846FDF726FF224602212846FDF784
:1045A00069FF02212846FDF73FFF0A480463012105
:1045B000417202212846FDF743FF054828388168EB
:1045C0008022114381602046F8BD000000000240B7
:1045D00028380140140200200248016A491C016287
:1045E000704700001402002010B50A48407A0028E5
:1045F0000DD1084C206F5834002808D12046FCF714
:1046000093F90146E26820688018FFF7B5FF0020A3
:1046100010BD000014020020F8B5144D0C460646EB
:1046200005212846FDF7F4FE002000903346104A8D
:1046300005212846FDF7D6FE224605212846FDF72E
:1046400019FF05212846FDF7EFFE0A4844630121C2
:10465000817205212846FDF7F3FE0548243881685C
:104660004022114381600020F8BD0000000002409C
:1046700024440040A80200200A480B490079405811
:10468000802180B2081A0949012208600849CA67D6
:104690004A6A521C4A62002803DD012005490007CE
:1046A00048607047CC5300080400024040000020DE
:1046B000A802002000ED00E0F8B5144D0C460646B7
:1046C00004212846FDF7A4FE10200090104B32462E
:1046D00004212846FDF786FE224604212846FDF7E0
:1046E000C9FE04212846FDF79FFE0A480463012104
:1046F000417204212846FDF7A3FE05482838816849
:104700008022114381602046F8BD00000000024075
:1047100028440040A80200200248016A491C0162A6
:1047200070470000A802002010B5054C0A466388B7
:1047300021465B1C4380FBF741FF002010BD0000B9
:10474000007C000870B50C460B494118002B08D0BE
:104750000A4D4519012B03D0094B9B8A002B00D130
:1047600029468005204603D000F042F8002070BDA5
:10477000FBF724FFFAE700000080000800A0000813
:10478000A8140020F8B54188174A491C41801549F2
:1047900001807E2100250A52ED438023002211462C
:1047A000124C002659430C19314603E0675CFF2F79
:1047B00004D1491C9942F9DB002E03D0521C082A6F
:1047C000EDDB00E01546082D06D208495D43691867
:1047D000802200F00DF803E080220449FBF7EEFE92
:1047E0000020F8BDAA550000A55A000000C000082E
:1047F000F7B50D460646FCF7F7F90298002487083E
:1048000007E0A0003258411900230220FCF7AEF95E
:10481000641CA742F5D802987C00470807E06000B6
:10482000325A411900230120FCF7A0F9641CA74269
:10483000F5D8FCF791F9FEBDFEE700000FB410B506
:1048400004A9074B02AA039800F028F8044602A91D
:10485000002000F05DFA204610BC08BC04B01847E8
:10486000114D000830B47446641E2578641CAB42B8
:1048700000D21D46635D5B00E31830BC184702E0C0
:1048800008C8121F08C1002AFAD1704770470020DB
:1048900001E001C1121F002AFBD17047FFB591B0A2
:1048A0000F460546002606E025280AD0149A1399DB
:1048B00090476D1C761C28780028F5D1304615B03D
:1048C000F0BD002400940121F34A029400E0044367
:1048D0006D1C2B780846203B98401042F7D1287871
:1048E0002A280ED0022128780246303A092A15D803
:1048F000009A0A235A43303A80180C436D1C0090EA
:10490000F1E701CF0090002805DA012040030443BD
:10491000009840420090022004436D1C28782E2805
:1049200015D10420044368786D1C2A280AD101CFD0
:104930006D1C02900BE002990A2251433039401855
:104940006D1C02902878014630390929F3D928785E
:104950006C2810D006DC4C281AD068280ED06A28A3
:1049600017D104E0742813D07A2812D110E0012066
:10497000400504430CE00121090501E0032109057C
:104980000C436978814203D10120000524186D1C75
:104990006D1C287803906E281ED00CDC632831D063
:1049A00004DC00288AD0582811D1B2E064287BD0DA
:1049B00069280CD178E073282DD004DC6F2870D0E2
:1049C000702804D1A7E075286CD078286BD0149A91
:1049D00013999047761C62E06002400F022807D0CE
:1049E00003280AD0042838680AD006603F1D56E024
:1049F0003868F11706604160F8E738680680F5E727
:104A00000670F3E73878694608740020487404A8F3
:104A10000390012003E0386803900020C0433F1D4D
:104A200061070FD5002101E00199491C029A01910B
:104A3000914213DA8142F7DB019A0399895C0029DC
:104A4000F2D10BE0002101E00199491C0191814262
:104A5000FADB019A0399895C0029F5D10199009844
:104A6000139A401A00902146149B00F03BF90199DB
:104A70008019461807E0039803990078491C0391B0
:104A8000149A139990470198401E0190401CF2D14E
:104A90002146149B139A009800F014F986196D1C96
:104AA00009E741E033E034E00A2000210490059159
:104AB0006002410F022905D001CFC2179446032995
:104AC00005D007E0FF1DFF08FF0003CF06E000B29E
:104AD000C2179446042902D140B2C1178C46002265
:104AE0006146944506DA0A460021404291418C46CF
:104AF0002D2102E0210504D52B216A4611760121E2
:104B000003E0E10701D02021F7E7019154E00A20FA
:104B10000BE0102009E01020049000210420044341
:104B200008200591029003E00820002105910490DF
:104B30006002410F022905D001CF002294460329CB
:104B400006D006E0FF1DFF08FF0003CF8C4603E000
:104B500080B2042900D1C0B20021019121072BD5D8
:104B60000399702906D0049A1021059B4A401A43E4
:104B700005D00EE040216A461176012108E0614629
:104B8000014306D030216A461176039951760221FD
:104B90000191049A0821059B4A401A430CD16146B1
:104BA000014301D1610707D530216A461176012101
:104BB00001910299491E02910399582904D037A105
:104BC00003910FA90F910DE039A1F9E76146059B0B
:104BD000049AFBF718FB039B8C469B5C0F9A521EB2
:104BE0000F92137061460143F0D10F9807A9081A7C
:104BF00020300390600704D501200004844302980C
:104C000001E0012002900399884201DD401A00E092
:104C1000002041180290019809180098401A00904D
:104C2000E00306D42146149B139A009800F05AF82A
:104C300086190020049008E006A9085C149A1399CC
:104C400090470498401C761C049001998842F3DB3D
:104C5000E0030CD52146149B139A009800F042F80B
:104C6000861904E0149A302013999047761C029913
:104C7000481E02900029F5DC08E00F980F99007893
:104C8000491C0F91149A13999047761C0399481E5A
:104C900003900029F1DCFBE60928010030313233B2
:104CA0003435363738396162636465660000000068
:104CB0003031323334353637383941424344454652
:104CC00000000000F8B5044600251E46174688047B
:104CD00004D405E039462020B0476D1C641EF9D588
:104CE0002846F8BDFFB50446002581B01E46C8031E
:104CF00001D5302700E02027880404D505E0384698
:104D00000399B0476D1C641EF9D5284605B0F0BD67
:104D10000A68531C0B6010707047000010B50A2120
:104D200001A0FEF7E1FE10BD1B5B324A1B5B303B6E
:104D30003048000030B503460B48002900D101215E
:104D40000A4C491E0ED31A7850400022C50702D0E3
:104D50004008604000E04008521CD2B2082AF5D357
:104D60005B1CEEE730BD0000FFFF000001A000006B
:104D700070B50A4DFF23EE1D1A46F93605E004789A
:104D800054402A5D5A40335D401C0C46491E89B28E
:104D9000002CF4D11802104370BD0000D255000859
:104DA00070B504460C4800220C4E11E02378521CCA
:104DB0001D4645402D07ED0E755B0009454018095D
:104DC00068400007C00E305A2B09584092B2641C4C
:104DD0008A42EBD370BD0000FFFF0000D2570008ED
:104DE00010B5084A084B07E0047854402406E40D47
:104DF0001C5B120A6240401C491EF5D2D04380B2AF
:104E000010BD0000FFFF0000D253000806C00021C3
:104E1000016041608160C160012202614161084618
:104E200070470000074910B54A8D0B464C3BD054E3
:104E3000488D401C80B24885642801D351204885A4
:104E400010BD000074140020F84F88B00126FF2028
:104E50003E830530F64B80220090991AF548FCF706
:104E6000DBFA4020F44B0246191A0090F348FCF795
:104E7000D3FAFBF7D9FE0021F14A0D4660204843E2
:104E8000801845608560056145618561C561056281
:104E900085624562C562491C05630929EEDBE94C60
:104EA000E9482567C06A6066E8480068A066E84887
:104EB000406AE066FFF75AFAE749E6480860FCF7FF
:104EC000BBFAFDF7F9FCFDF7E3FCFDF72FFAE34829
:104ED000FEF79EFED5480683FEF792FE1021A063E2
:104EE00008430107090F6063DD4AC006DD48117001
:104EF00003D50670DC48057002E00570DA480670DC
:104F0000DA480170FBF704FCD54801270178D7483F
:104F10000170D748D7490770E12080020860FDF78B
:104F20000FFEFDF79FFEFDF77BFDD348416840264D
:104F300031434160FDF75AFDFDF7D8FDCF480168C8
:104F400039430160CE4801682022114301600168A5
:104F50001027394301600168314301608021C9484D
:104F6000FFF75AFBC84801683943016001683143C3
:104F700001600A20FBF792FD0120FFF745F80020B1
:104F8000FFF72AF80020FFF733F8FFF7ADF8FBF73B
:104F90006FFDA64F60663D827D82B048C088388232
:104FA000388A01280AD1FCF7F1F9208F2021084026
:104FB0007882788A002801D0FFF758F9B34E5A203A
:104FC0007084B3480690B34D00272F70012068709D
:104FD000FBF74EFD2861FBF719FE0790FEF710FE68
:104FE00005469248008AC0070BD0A806208F04D53A
:104FF000800606D4FFF73AF903E0800601D5FFF7F3
:105000006DF9A5630798E0630920C0060069069959
:105010008884A1480069C884A04800690885A04820
:1050200000694885FBF798FBFBF722FD994D686105
:105030009C480068002800D0B782206CC006C00ED3
:1050400002281BD1FBF732F99648016800290DD0E0
:105050009549B7820A68002A10D100680860934811
:10506000006893490860FEF7B5F907E08E490A68C1
:10507000002A03D000680860FEF7C4F96B48008A74
:1050800001280BD16948818A00291FD08949A9606C
:10509000C18A89480160A868FEF7BCF9606E696939
:1050A0006166081AA066E16E884200D2E066216F50
:1050B000884200D92067FBF7DBFCA86169480078CB
:1050C000002818D07D4900200B780BE07C49DEE7F2
:1050D0007C4913220918520189180A7D7A49091856
:1050E0004A70401C9842F3DB60480078002802D0E8
:1050F0000220FCF799FA0798800402D50120287055
:1051000000E02F700798000502D50120687000E0CC
:105110006F7055480078002819D00220FCF760FC19
:10512000606C002801D169480770684868490078B8
:10513000B0860868800402D50120287000E02F7036
:105140000868000502D50120687000E06F70606C8F
:10515000002801D0401E6064A06C002801D0401ED1
:10516000A0643248018B002946D06878FEF74CFFD6
:105170006878FEF731FF6878FEF722FF687800282C
:1051800001D1012000E00020FEF732FFFBF770FCA8
:10519000E8615049B08A888608464030808AB086E7
:1051A000FBF766FC2862FBF763FC0A21686208468D
:1051B000FAF78AFF0020401C4028FCDB206C46499F
:1051C000401C2064086800282FDD1A4AD26F002A8C
:1051D0002BD082B241490120FDF70CFE002805D0FA
:1051E0003D483E4902680120FCF710FD3A4807603F
:1051F0001048C7676F6091E0008A01280FD0606C8B
:10520000002810D06878FEF7FFFEA06C00286AD056
:105210006878FEF7E1FE6878FEF7D2FEB3E7304823
:1052200000680028EFD02878EDE763E0A81400209C
:10523000A815002014020020EC160020A80200206F
:105240005C0500207412002080F7FF1F3000002052
:10525000001002401027000014000020740C0020F1
:10526000500000204C0000204D000020570000207E
:1052700051000020340000200030014000100040A8
:1052800000380140BC03002000440040340F0020DF
:1052900074140020E40000200004004800080048C6
:1052A000000C0048BC000020C000002018000020B6
:1052B000C400002000A0000894000020CB000020C3
:1052C00000800008F40C00204C0400203C04002066
:1052D00068000020B41000203C0000203C030020A7
:1052E0006C0A0020FFE70020FEF776FE0020FEF7A4
:1052F00067FE46E72849686888420DD92748416813
:1053000001221205114341604168520003235B05ED
:1053100099431143416001E0401C686020480078D7
:10532000002802D00020FBF7B9FB18221D4968466F
:10533000FAF73BFF1C4D00206F461C4942005118F4
:1053400040310A891105130B1207090E120F0029AB
:1053500018D0002B02D0012B06D013E0144B5918A3
:1053600009239B01C91804E0114B5B181321490163
:105370005918C97C01239340194203D08100795800
:10538000A96102E081007958A962401C0628D4DB9B
:1053900009490848086016E6C0270900003801409E
:1053A0004D000020A858000800040048740C00209C
:1053B000F40C0020AAAA000000300040112233445F
:1053C0005566778899AABBCCDDEEFF00081C3044F7
:1053D00058000000891112239B322446AD573665D0
:1053E000BF74488CC19D5AAFD3BE6CCAE5DB7EE961
:1053F000F7F88110080193331A22A5562C47B77588
:105400003E64C99C408DDBBF52AEEDDA64CBFFF940
:1054100076E802218B30100299132667AF76344468
:10542000BD554AADC3BC588ED19F6EEBE7FA7CC820
:10543000F5D983310A2091121803A7772E66B55447
:105440003C45CBBD42ACD99E508FEFFB66EAFDD800
:1054500074C904428D5316619F702004A915322728
:10546000BB364CCEC5DF5EEDD7FC6888E1997AABE0
:10547000F3BA85520C4397711E60A1142805B33707
:105480003A26CDDE44CFDFFD56ECE9986089FBBBC0
:1054900072AA06638F7214409D512225AB343006E8
:1054A000B9174EEFC7FE5CCCD5DD6AA9E3B8788AA0
:1054B000F19B87730E6295501C41A3352A24B116C7
:1054C0003807CFFF46EEDDDC54CDEBB962A8F99A80
:1054D000708B088481951AA793B62CC2A5D33EE1A0
:1054E000B7F04008C919522BDB3A644EED5F766D78
:1054F000FF7C899400859BB712A6ADD224C3BFF16F
:1055000036E0C1184809D33B5A2AE55E6C4FF77D57
:105510007E6C0AA583B4188691972EE3A7F23CC04F
:10552000B5D14229CB38500AD91B666FEF7E744C37
:10553000FD5D8BB502A499961087AFF326E2BDD02E
:1055400034C1C3394A28D11A580BE77F6E6EF55C17
:105550007C4D0CC685D71EE597F42880A1913AA30F
:10556000B3B2444ACD5B5669DF78600CE91D722FF7
:10557000FB3E8DD604C79FF516E4A9902081BBB3EE
:1055800032A2C55A4C4BD7795E68E11C680DF33FD7
:105590007A2E0EE787F61CC495D52AA1A3B03882CF
:1055A000B193466BCF7A5448DD59622DEB3C700EB7
:1055B000F91F8FF706E69DD414C5ABB122A0B992AE
:1055C0003083C77B4E6AD5585C49E33D6A2CF11E97
:1055D000780F00C1814001C0804101C0804100C1FD
:1055E000814001C0804100C1814000C1814001C0B3
:1055F000804101C0804100C1814000C1814001C0A3
:10560000804100C1814001C0804101C0804100C192
:10561000814001C0804100C1814000C1814001C082
:10562000804100C1814001C0804101C0804100C172
:10563000814000C1814001C0804101C0804100C162
:10564000814001C0804100C1814000C1814001C052
:10565000804101C0804100C1814000C1814001C042
:10566000804100C1814001C0804101C0804100C132
:10567000814000C1814001C0804101C0804100C122
:10568000814001C0804100C1814000C1814001C012
:10569000804100C1814001C0804101C0804100C102
:1056A000814001C0804100C1814000C1814001C0F2
:1056B000804101C0804100C1814000C1814001C0E2
:1056C000804100C1814001C0804101C0804100C1D2
:1056D000814000C0C101C30302C2C60607C705C599
:1056E000C404CC0C0DCD0FCFCE0E0ACACB0BC9090A
:1056F00008C8D81819D91BDBDA1A1EDEDF1FDD1D1A
:105700001CDC14D4D515D71716D6D21213D311D149
:10571000D010F03031F133F3F23236F6F737F53599
:1057200034F43CFCFD3DFF3F3EFEFA3A3BFB39F9C9
:10573000F83828E8E929EB2B2AEAEE2E2FEF2DED99
:10574000EC2CE42425E527E7E62622E2E323E12109
:1057500020E0A06061A163A3A26266A6A767A56519
:1057600064A46CACAD6DAF6F6EAEAA6A6BAB69A989
:10577000A86878B8B979BB7B7ABABE7E7FBF7DBD99
:10578000BC7CB47475B577B7B67672B2B373B171C9
:1057900070B0509091519353529296565797559599
:1057A00094549C5C5D9D5F9F9E5E5A9A9B5B995949
:1057B0005898884849894B8B8A4A4E8E8F4F8D4D19
:1057C0004C8C448485458747468682424383418189
:1057D0008040000001CC01D8001401F0003C0028FA
:1057E00001E401A0006C007801B40050019C018824
:1057F0000044030E04010001000104010006000042
:10580000000000000000000006000000AA55000093
:10581000000100000000000001000100000900007C
:10582000000000000000020000000009000000006D
:105830000000000000000000000000000000000068
:105840000000000010101010101010101010101098
:1058500010101010100020003000400050006000B8
:105860000300000004000000050000000600000026
:105870000700000008000000090000000A00000006
:105880000B0000000C0000001100A55AAA550000F2
:10589000000000000000000000000000081C304470
:1058A00058081C30445800000004000000080000A4
:1058B00000100000002000000040000000800000F8
:1058C00000000000000000000102030406070809B0
:1058D0000000000001020304F85800080000002046
:1058E000140100007E4800080C5A00081401002032
:1058F0003C1A00008E480008000000000000000074
:10590000000000000000000001000000102700005F
:105910000000000000000000000000000000000087
:1059200000000000000000000000000000840300F0
:1059300040420F00000000000000000000000000D6
:105940000000000000000100000000010101000053
:105950000000000000000000000000000000000047
:105960000000000000000000000000000000000037
:105970000000000000000000000000000100000026
:10598000000000000000000001000000970000007F
:10599000FFFFFFFF0000000000000000000000000B
:1059A00000000000000000000000000000000000F7
:1059B00000000000000000000000000000000000E7
:1059C00000000808000000000000000000000000C7
:1059D00000000000000000000000000000000000C7
:1059E000000000000080000800000000000000002F
:1059F00000000000000000000000000000000000A7
:0C5A000000000000001BB70000000000C8
:04000005080000B53A
:00000001FF
